:1000000000308A0004280000FF238316900000308F
:100010008A00892830308400000803191D28013027
:10002000A100A001A00B1228A10B11284A30A000AA
:10003000A00B18281B28800B0F280800831685109A
:1000400083128510831605108312051083168515FB
:1000500085128312851683160512831205128316E4
:10006000051583129D28A4010230A500A601A70151
:100070009830A8008830A9007F30AA009E28051279
:100080000130B0000A2005160A30B0000A209F286F
:10009000B30803194D2805144E28051000008514D7
:1000A0000000851008008512B3014820B3014820E4
:1000B0000130B3004820B3014820B3014820B30108
:1000C0004820B3014820B3014820B2013208073C60
:1000D000031C7628B01F70280130B3004820722816
:1000E000B30148200310B00DB20A6628B2013208ED
:1000F000073C031C8728B11F81280130B30048202A
:100100008328B30148200310B10DB20A7728851661
:10011000080084011F3083051F1383161F109F10D2
:100120001F119F11073083129900FF30831685003D
:10013000C8308312B0000A201E2833283F28B0019F
:100140002408B10053200130B0002508B10053202D
:100150000230B0002608B10053200330B000270859
:10016000B10053200430B0002808B10053200530FE
:10017000B0002908B10053200630B0002A08B100B1
:100180005320051DC6289830AE00C8289030AE0018
:1001900028082E020319D3282E08A8000430B00026
:0A01A0002808B1005320C1286300B5
:02400E00043F6D
:00000001FF
